:03000000020600F5
:03000300021A03DB
:03000B00021A06D0
:03001300021A09C5
:03001B00021A0CBA
:03002300021A0FAF
:03002B00021A12A4
:03003300021A1599
:03003B00021A188E
:03004300021A1B83
:03004B00021A1E78
:03005300021A216D
:03005B00021A2462
:03006300021A2757
:03006B00021A2A4C
:03007300021A2D41
:10060000E4F5D9E5EF7480F5FF7402F5EF787FE447
:10061000F6D8FD9000007F007E08E4F0A3DFFCDE4A
:07062000FA75812202066257
:1006A7000800080308060809080C080F08120815AF
:1006B7000819081C081F082208250828082B082FD6
:1006C700083208350838083B083E084108450848FD
:1006D700084B084E085108540857085B085E086124
:1006E70008640867086A086D087108740877087A4B
:1006F700087D088008830886088A088D0890089373
:1007070008960899089C08A008A308A608A908AC99
:1007170008AF08B208B508B908BC08BF08C208C5C1
:1007270008C808CB08CE08D208D508D808DB08DEE9
:1007370008E108E408E708EB08EE08F108F408F711
:1007470008FA08FD090009040907090A090D091033
:10075700091309160919091C09200923092609295A
:10076700092C092F093209350938093C093F094283
:1007770009450948094B094E095109540957095BAD
:10078700095E096109640967096A096D09700973D6
:1007970009760979097D0980098309860989098C00
:1007A700098F099209950998099B099E09A209A52C
:1007B70009A809AB09AE09B109B409B709BA09BD56
:1007C70009C009C309C609C909CC09D009D309D683
:1007D70009D909DC09DF09E209E509E809EB09EEAE
:1007E70009F109F409F709FA09FD0A000A030A06DB
:1007F7000A090A0D0A100A130A160A190A1C0A1FFF
:100807000A220A250A280A2B0A2E0A310A340A372D
:100817000A3A0A3D0A400A430A460A490A4C0A4F5D
:100827000A520A550A580A5B0A5E0A610A640A678D
:100837000A6A0A6D0A700A730A760A790A7C0A7FBD
:100847000A820A850A880A8B0A8E0A910A940A97ED
:100857000A9A0A9D0AA00AA30AA60AA90AAC0AAE1E
:100867000AB10AB40AB70ABA0ABD0AC00AC30AC655
:100877000AC90ACC0ACF0AD20AD50AD80ADB0ADE85
:100887000AE10AE30AE60AE90AEC0AEF0AF20AF5BC
:100897000AF80AFB0AFE0B010B040B070B090B0CEA
:1008A7000B0F0B120B150B180B1B0B1E0B210B241D
:1008B7000B260B290B2C0B2F0B320B350B380B3B55
:1008C7000B3D0B400B430B460B490B4C0B4F0B518E
:1008D7000B540B570B5A0B5D0B600B630B650B68C7
:1008E7000B6B0B6E0B710B740B760B790B7C0B7F01
:1008F7000B820B850B870B8A0B8D0B900B930B953C
:100907000B980B9B0B9E0BA10BA40BA60BA90BAC77
:100917000BAF0BB10BB40BB70BBA0BBD0BBF0BC2B5
:100927000BC50BC80BCA0BCD0BD00BD30BD60BD8F3
:100937000BDB0BDE0BE10BE30BE60BE90BEB0BEE33
:100947000BF10BF40BF60BF90BFC0BFF0C010C0472
:100957000C070C090C0C0C0F0C120C140C170C1AAE
:100967000C1C0C1F0C220C240C270C2A0C2D0C2FF2
:100977000C320C350C370C3A0C3D0C3F0C420C4535
:100987000C470C4A0C4C0C4F0C520C540C570C5A7D
:100997000C5C0C5F0C620C640C670C690C6C0C6FC4
:1009A7000C710C740C770C790C7C0C7E0C810C840C
:1009B7000C860C890C8B0C8E0C900C930C960C9857
:1009C7000C9B0C9D0CA00CA20CA50CA80CAA0CADA2
:1009D7000CAF0CB20CB40CB70CB90CBC0CBE0CC1F0
:1009E7000CC30CC60CC90CCB0CCE0CD00CD30CD53D
:1009F7000CD80CDA0CDD0CDF0CE20CE40CE70CE98C
:100A07000CEB0CEE0CF00CF30CF50CF80CFA0CFDDF
:100A17000CFF0D020D040D070D090D0B0D0E0D102A
:100A27000D130D150D180D1A0D1C0D1F0D210D247D
:100A37000D260D280D2B0D2D0D300D320D340D37D4
:100A47000D390D3C0D3E0D400D430D450D470D4A2B
:100A57000D4C0D4E0D510D530D560D580D5A0D5D84
:100A67000D5F0D610D640D660D680D6A0D6D0D6FDF
:100A77000D710D740D760D780D7B0D7D0D7F0D813C
:100A87000D840D860D880D8A0D8D0D8F0D910D949A
:100A97000D960D980D9A0D9D0D9F0DA10DA30DA5FA
:100AA7000DA80DAA0DAC0DAE0DB10DB30DB50DB75B
:100AB7000DB90DBC0DBE0DC00DC20DC40DC60DC9BF
:100AC7000DCB0DCD0DCF0DD10DD30DD60DD80DDA24
:100AD7000DDC0DDE0DE00DE20DE50DE70DE90DEB8B
:100AE7000DED0DEF0DF10DF30DF50DF70DFA0DFCF5
:100AF7000DFE0E000E020E040E060E080E0A0E0C58
:100B07000E0E0E100E120E140E160E180E1B0E1DC4
:100B17000E1F0E210E230E250E270E290E2B0E2D2E
:100B27000E2F0E310E330E350E370E390E3B0E3C9F
:100B37000E3E0E400E420E440E460E480E4A0E4C16
:100B47000E4E0E500E520E540E560E580E5A0E5B87
:100B57000E5D0E5F0E610E630E650E670E690E6BFE
:100B67000E6C0E6E0E700E720E740E760E780E7977
:100B77000E7B0E7D0E7F0E810E830E840E860E88F1
:100B87000E8A0E8C0E8E0E8F0E910E930E950E966C
:100B97000E980E9A0E9C0E9E0E9F0EA10EA30EA5EA
:100BA7000EA60EA80EAA0EAC0EAD0EAF0EB10EB26B
:100BB7000EB40EB60EB80EB90EBB0EBD0EBE0EC0ED
:100BC7000EC20EC30EC50EC70EC80ECA0ECC0ECD72
:100BD7000ECF0ED10ED20ED40ED60ED70ED90EDBF7
:100BE7000EDC0EDE0EDF0EE10EE30EE40EE60EE780
:100BF7000EE90EEA0EEC0EEE0EEF0EF10EF20EF40B
:100C07000EF50EF70EF90EFA0EFC0EFD0EFF0F0095
:100C17000F020F030F050F060F080F090F0B0F0C1D
:100C27000F0E0F0F0F110F120F140F150F160F18AE
:100C37000F190F1B0F1C0F1E0F1F0F210F220F2342
:100C47000F250F260F280F290F2A0F2C0F2D0F2FD7
:100C57000F300F310F330F340F350F370F380F3A6F
:100C67000F3B0F3C0F3E0F3F0F400F420F430F4408
:100C77000F450F470F480F490F4B0F4C0F4D0F4FA5
:100C87000F500F510F520F540F550F560F570F5943
:100C97000F5A0F5B0F5C0F5E0F5F0F600F610F62E4
:100CA7000F640F650F660F670F680F6A0F6B0F6C86
:100CB7000F6D0F6E0F6F0F710F720F730F740F752C
:100CC7000F760F770F790F7A0F7B0F7C0F7D0F7ED3
:100CD7000F7F0F800F810F820F840F850F860F877D
:100CE7000F880F890F8A0F8B0F8C0F8D0F8E0F8F29
:100CF7000F900F910F920F930F940F950F960F97D9
:100D07000F980F990F9A0F9B0F9C0F9D0F9E0F9F88
:100D17000FA00FA10FA20FA30FA40FA50FA50FA63A
:100D27000FA70FA80FA90FAA0FAB0FAC0FAD0FAEF0
:100D37000FAE0FAF0FB00FB10FB20FB30FB40FB4A9
:100D47000FB50FB60FB70FB80FB90FB90FBA0FBB63
:100D57000FBC0FBD0FBD0FBE0FBF0FC00FC10FC11F
:100D67000FC20FC30FC40FC40FC50FC60FC70FC7DE
:100D77000FC80FC90FCA0FCA0FCB0FCC0FCC0FCD9F
:100D87000FCE0FCE0FCF0FD00FD00FD10FD20FD264
:100D97000FD30FD40FD40FD50FD60FD60FD70FD829
:100DA7000FD80FD90FD90FDA0FDB0FDB0FDC0FDCF2
:100DB7000FDD0FDD0FDE0FDF0FDF0FE00FE00FE1BD
:100DC7000FE10FE20FE20FE30FE30FE40FE40FE58C
:100DD7000FE50FE60FE60FE70FE70FE80FE80FE95C
:100DE7000FE90FEA0FEA0FEB0FEB0FEC0FEC0FEC2D
:100DF7000FED0FED0FEE0FEE0FEF0FEF0FEF0FF001
:100E07000FF00FF00FF10FF10FF20FF20FF20FF3D8
:100E17000FF30FF30FF40FF40FF40FF50FF50FF5B2
:100E27000FF60FF60FF60FF70FF70FF70FF70FF88D
:100E37000FF80FF80FF80FF90FF90FF90FF90FFA6D
:100E47000FFA0FFA0FFA0FFB0FFB0FFB0FFB0FFB4E
:100E57000FFC0FFC0FFC0FFC0FFC0FFD0FFD0FFD30
:100E67000FFD0FFD0FFD0FFD0FFE0FFE0FFE0FFE17
:100E77000FFE0FFE0FFE0FFE0FFF0FFF0FFF0FFFFF
:100E87000FFF0FFF0FFF0FFF0FFF0FFF0FFF0FFFEB
:100E97000FFF0FFF0FFF0FFF0FFF0FFF0FFF0FFFDB
:100EA7000FFF0FFF0FFF0FFF0FFF0FFF0FFF0FFFCB
:100EB7000FFF0FFF0FFF0FFF0FFF0FFF0FFF0FFFBB
:100EC7000FFF0FFF0FFF0FFF0FFF0FFE0FFE0FFEAE
:100ED7000FFE0FFE0FFE0FFE0FFE0FFD0FFD0FFDA6
:100EE7000FFD0FFD0FFD0FFD0FFC0FFC0FFC0FFC9F
:100EF7000FFC0FFB0FFB0FFB0FFB0FFB0FFA0FFA9C
:100F07000FFA0FFA0FF90FF90FF90FF90FF80FF89A
:100F17000FF80FF80FF70FF70FF70FF70FF60FF69A
:100F27000FF60FF50FF50FF50FF40FF40FF40FF39E
:100F37000FF30FF30FF20FF20FF20FF10FF10FF0A4
:100F47000FF00FF00FEF0FEF0FEF0FEE0FEE0FEDAC
:100F57000FED0FEC0FEC0FEC0FEB0FEB0FEA0FEAB7
:100F67000FE90FE90FE80FE80FE70FE70FE60FE6C6
:100F77000FE50FE50FE40FE40FE30FE30FE20FE2D6
:100F87000FE10FE10FE00FE00FDF0FDF0FDE0FDDE7
:100F97000FDD0FDC0FDC0FDB0FDB0FDA0FD90FD9FB
:100FA7000FD80FD80FD70FD60FD60FD50FD40FD412
:100FB7000FD30FD20FD20FD10FD00FD00FCF0FCE2D
:100FC7000FCE0FCD0FCC0FCC0FCB0FCA0FCA0FC947
:100FD7000FC80FC70FC70FC60FC50FC40FC40FC366
:100FE7000FC20FC10FC10FC00FBF0FBE0FBD0FBD87
:100FF7000FBC0FBB0FBA0FB90FB90FB80FB70FB6AA
:101007000FB50FB40FB40FB30FB20FB10FB00FAFCF
:101017000FAE0FAE0FAD0FAC0FAB0FAA0FA90FA8F6
:101027000FA70FA60FA50FA50FA40FA30FA20FA120
:101037000FA00F9F0F9E0F9D0F9C0F9B0F9A0F994D
:101047000F980F970F960F950F940F930F920F917D
:101057000F900F8F0F8E0F8D0F8C0F8B0F8A0F89AD
:101067000F880F870F860F850F840F820F810F80E0
:101077000F7F0F7E0F7D0F7C0F7B0F7A0F790F7716
:101087000F760F750F740F730F720F710F6F0F6E4F
:101097000F6D0F6C0F6B0F6A0F680F670F660F6589
:1010A7000F640F620F610F600F5F0F5E0F5C0F5BC6
:1010B7000F5A0F590F570F560F550F540F520F5105
:1010C7000F500F4F0F4D0F4C0F4B0F490F480F4746
:1010D7000F450F440F430F420F400F3F0F3E0F3C8A
:1010E7000F3B0F3A0F380F370F350F340F330F31D0
:1010F7000F300F2F0F2D0F2C0F2A0F290F280F2618
:101107000F250F230F220F210F1F0F1E0F1C0F1B61
:101117000F190F180F160F150F140F120F110F0FAE
:101127000F0E0F0C0F0B0F090F080F060F050F03FC
:101137000F020F000EFF0EFD0EFC0EFA0EF90EF752
:101147000EF50EF40EF20EF10EEF0EEE0EEC0EEAA9
:101157000EE90EE70EE60EE40EE30EE10EDF0EDEFD
:101167000EDC0EDB0ED90ED70ED60ED40ED20ED154
:101177000ECF0ECD0ECC0ECA0EC80EC70EC50EC3AF
:101187000EC20EC00EBE0EBD0EBB0EB90EB80EB609
:101197000EB40EB20EB10EAF0EAD0EAC0EAA0EA867
:1011A7000EA60EA50EA30EA10E9F0E9E0E9C0E9AC6
:1011B7000E980E960E950E930E910E8F0E8E0E8C28
:1011C7000E8A0E880E860E840E830E810E7F0E7D8C
:1011D7000E7B0E790E780E760E740E720E700E6EF2
:1011E7000E6C0E6B0E690E670E650E630E610E5F59
:1011F7000E5D0E5B0E5A0E580E560E540E520E50C2
:101207000E4E0E4C0E4A0E480E460E440E420E402F
:101217000E3E0E3C0E3B0E390E370E350E330E3199
:101227000E2F0E2D0E2B0E290E270E250E230E2107
:101237000E1F0E1D0E1B0E180E160E140E120E107C
:101247000E0E0E0C0E0A0E080E060E040E020E00EF
:101257000DFE0DFC0DFA0DF70DF50DF30DF10DEF6C
:101267000DED0DEB0DE90DE70DE50DE20DE00DDEE2
:101277000DDC0DDA0DD80DD60DD30DD10DCF0DCD5B
:101287000DCB0DC90DC60DC40DC20DC00DBE0DBCD5
:101297000DB90DB70DB50DB30DB10DAE0DAC0DAA52
:1012A7000DA80DA50DA30DA10D9F0D9D0D9A0D98D0
:1012B7000D960D940D910D8F0D8D0D8A0D880D8650
:1012C7000D840D810D7F0D7D0D7B0D780D760D74D1
:1012D7000D710D6F0D6D0D6A0D680D660D640D6155
:1012E7000D5F0D5D0D5A0D580D560D530D510D4ED9
:1012F7000D4C0D4A0D470D450D430D400D3E0D3C60
:101307000D390D370D340D320D300D2D0D2B0D28E8
:101317000D260D240D210D1F0D1C0D1A0D180D1571
:101327000D130D100D0E0D0B0D090D070D040D02FC
:101337000CFF0CFD0CFA0CF80CF50CF30CF00CEE92
:101347000CEB0CE90CE70CE40CE20CDF0CDD0CDA1F
:101357000CD80CD50CD30CD00CCE0CCB0CC90CC6AE
:101367000CC30CC10CBE0CBC0CB90CB70CB40CB242
:101377000CAF0CAD0CAA0CA80CA50CA20CA00C9DD4
:101387000C9B0C980C960C930C900C8E0C8B0C8968
:101397000C860C840C810C7E0C7C0C790C770C74FD
:1013A7000C710C6F0C6C0C690C670C640C620C5F95
:1013B7000C5C0C5A0C570C540C520C4F0C4C0C4A2E
:1013C7000C470C450C420C3F0C3D0C3A0C370C35C6
:1013D7000C320C2F0C2D0C2A0C270C240C220C1F62
:1013E7000C1C0C1A0C170C140C120C0F0C0C0C09FF
:1013F7000C070C040C010BFF0BFC0BF90BF60BF4A1
:101407000BF10BEE0BEB0BE90BE60BE30BE10BDE42
:101417000BDB0BD80BD60BD30BD00BCD0BCA0BC8E2
:101427000BC50BC20BBF0BBD0BBA0BB70BB40BB184
:101437000BAF0BAC0BA90BA60BA40BA10B9E0B9B25
:101447000B980B950B930B900B8D0B8A0B870B85CA
:101457000B820B7F0B7C0B790B760B740B710B6E6E
:101467000B6B0B680B650B630B600B5D0B5A0B5714
:101477000B540B510B4F0B4C0B490B460B430B40BB
:101487000B3D0B3B0B380B350B320B2F0B2C0B2962
:101497000B260B240B210B1E0B1B0B180B150B120A
:1014A7000B0F0B0C0B090B070B040B010AFE0AFBB6
:1014B7000AF80AF50AF20AEF0AEC0AE90AE60AE369
:1014C7000AE10ADE0ADB0AD80AD50AD20ACF0ACC11
:1014D7000AC90AC60AC30AC00ABD0ABA0AB70AB4C1
:1014E7000AB10AAE0AAC0AA90AA60AA30AA00A9D6B
:1014F7000A9A0A970A940A910A8E0A8B0A880A8519
:101507000A820A7F0A7C0A790A760A730A700A6DC8
:101517000A6A0A670A640A610A5E0A5B0A580A5578
:101527000A520A4F0A4C0A490A460A430A400A3D28
:101537000A3A0A370A340A310A2E0A2B0A280A25D8
:101547000A220A1F0A1C0A190A160A130A100A0D88
:101557000A090A060A030A0009FD09FA09F709F444
:1015670009F109EE09EB09E809E509E209DF09DCF8
:1015770009D909D609D309D009CC09C909C609C3AC
:1015870009C009BD09BA09B709B409B109AE09AB60
:1015970009A809A509A2099E099B09980995099215
:1015A700098F098C0989098609830980097D0979C9
:1015B700097609730970096D096A09670964096180
:1015C700095E095B095709540951094E094B094836
:1015D70009450942093F093C093809350932092FEC
:1015E700092C0929092609230920091C09190916A3
:1015F70009130910090D090A09070904090008FD5B
:1016070008FA08F708F408F108EE08EB08E708E419
:1016170008E108DE08DB08D808D508D208CE08CBD1
:1016270008C808C508C208BF08BC08B908B508B289
:1016370008AF08AC08A908A608A308A0089C089941
:10164700089608930890088D088A088608830880FA
:10165700087D087A087708740871086D086A0867B2
:1016670008640861085E085B085708540851084E6B
:10167700084B084808450841083E083B0838083524
:101687000832082F082B082808250822081F081CDD
:10169700081908150812080F080C08090806080396
:1016A7001000100B10161021102C10371043104E7D
:1016B700105910651070107B10871092109E10A99A
:1016C70010B510C010CC10D810E310EF10FB1107A5
:1016D7001113111E112A11361142114E115A11669A
:1016E7001172117E118A119711A311AF11BB11C885
:1016F70011D411E011ED11F912061212121F122B5B
:10170700123812451251125E126B1278128412911E
:10171700129E12AB12B812C512D212DF12EC12F9D6
:10172700130613141321132E133C13491356136472
:101737001371137F138C139A13A713B513C313D005
:1017470013DE13EC13FA1408141614231431143F80
:10175700144E145C146A14781486149414A314B1E8
:1017670014BF14CE14DC14EB14F91508151615253F
:101777001534154215511560156F157E158D159C7D
:1017870015AB15BA15C915D815E715F616051615AB
:1017970016241633164316521662167116811690C2
:1017A70016A016B016C016CF16DF16EF16FF170FC6
:1017B700171F172F173F174F175F177017801790AF
:1017C70017A117B117C117D217E217F31804181486
:1017D700182518361847185718681879188A189B43
:1017E70018AC18BE18CF18E018F1190219141925EA
:1017F70019371948195A196B197D198F19A019B278
:1018070019C419D619E819FA1A0C1A1E1A301A42ED
:101817001A551A671A791A8B1A9E1AB01AC31AD54B
:101827001AE81AFB1B0E1B201B331B461B591B6C8C
:101837001B7F1B921BA51BB81BCC1BDF1BF21C06B7
:101847001C191C2D1C401C541C671C7B1C8F1CA3C3
:101857001CB71CCB1CDF1CF31D071D1B1D2F1D43B5
:101867001D581D6C1D801D951DA91DBE1DD31DE78F
:101877001DFC1E111E261E3B1E501E651E7A1E8F46
:101887001EA41EB91ECF1EE41EFA1F0F1F251F3AE6
:101897001F501F661F7B1F911FA71FBD1FD31FE967
:1018A7000C000B000A0009000800070006000500ED
:0C18B7000400030002000100010000001A
:102E7C004102864CC108C10BC10A410285004102C6
:102E8C008700C1894102960041023E01410297012F
:102E9C004202820001410284064102070042029470
:102EAC0000004202020000410204004202900001B4
:102EBC004202920000420288000042023F0001429E
:082ECC00020500004102810132
:10315800E4F5AB53E3DF75B61043E32075AB80FFAE
:10316800EFC394C850030F80F743ABC0E4FFEFC32D
:0F31780094C850030F80F7E5AB30E5FB75B287C5
:013187002225
:10338400758921758E0C758CFE758A1A7588307551
:0E339400C804E4F5CA75CBFEF5CC75CDFE225B
:1034250075BC90900284E0F5BB75E88075BAF7220B
:0734560075B9F675B5F62209
:04347700E4F5D12285
:1033A200E4F5F275A48075A63875D40375D5FF755A
:0B33B200F3FFF5D675E10475E2402240
:0A34440075B80275E60975A8A2220A
:10332500E4F5881231581233A2123384123425126F
:103335003456123477123444123233C2A5C20A22EB
:08327D00AB07AF031BEF601A61
:1032850090039F121C680000445C90039F74FF121A
:0A3295001C29EC4D4E4F60E280F062
:01329F00220C
:102E0200C21153D9BF123325A2A2921130110890D8
:102E12000286744CF08006900286744DF01233BD27
:102E22001232A0123188EF60FAC2AF900353E0B4BD
:102E32000B02D208900353E0B41407D209D20A124B
:102E420033EE900353E0B41504C20AC209300925D7
:102E5200900353E014601304701B900354E090033A
:102E6200A5F01232A0123401800B900354E09003BB
:092E7200A5F0121A1BD2AF80AAD0
:012E7B002234
:10340100A20A92A5E51424FFB392A4E51424FF9225
:02341100A322F4
:102C1E00900296E090023EF0E5805440900296F0CD
:102C2E00E07036900203E004F07006900202E004B9
:102C3E00F0D3900203E09400900202E09406404824
:102C4E00900286E0FF7D081233049002047401F0B6
:102C5E00E4900202F0A3F0802FE4900202F0A3F0C1
:102C6E0090023EE0701D900204E07017900297E013
:102C7E0070047F0180027F00900297EFF0E0F51460
:102C8E001233EEE4900204F0900285E0900287F099
:102C9E00E5A05402900285F0900287E06022900237
:102CAE0085E0701C900287F020080C9003A5F012AE
:102CBE001A1BC20BC20A22A209B39209A209920AD6
:012CCE0022E3
:031A060002307833
:10307800C0E0C0F0C083C082C0D075D000C000C01E
:1030880001C002C003C004C005C006C007122A3828
:10309800758CFE758A1AD007D006D005D004D003E7
:1030A800D002D001D000D0D0D082D083D0F0D0E0F0
:0130B80032E5
:102A3800900288E0A3E0F596900292E0A3E0F5F416
:102A4800900288E0F597900292E0F5F590023FE059
:102A5800FEA3E0FF900206E02FF0900205E03EF0B2
:102A6800E0C4F854F0C868FEA3E0C4540F48FFEE71
:102A7800540FAD07FCE42DFFEC3404AB07FA540FF8
:102A8800FAC3EC648094885021ED25E0FFEC33FE16
:102A980074A72FF58274063EF583E493FF740193BF
:102AA800900288CFF0A3EFF0802BEC5407FEED25C1
:102AB800E0FFEE33FE74A72FF58274063EF583E43B
:102AC80093FE740193FFC374FF9F900289F0740F03
:102AD8009E900288F0C3EA648094885020EB25E039
:102AE800FFEA33FE74A72FF58274063EF583E4935C
:102AF800FF740193900292CFF0A3EFF022EA5407FB
:102B0800FEEB25E0FFEE33FE74A72FF58274063E38
:102B1800F583E493FE740193FFC374FF9F900293BF
:082B2800F0740F9E900292F080
:012B30002282
:031A12000219C8EE
:1019C800C0E0C0F0C083C082C0D075D000C000C0E5
:1019D80001C002C003C004C005C006C00753C87FC9
:1019E8001232C2D007D006D005D004D003D002D01E
:0E19F80001D000D0D0D082D083D0F0D0E03229
:1032C200900284E0F5BBE004F0E0D36480948F4088
:1032D2000C7406F012340112345D12211643E81008
:0132E20022C9
:07345D00E51424FF92872211
:031A2100022EE6AC
:102EE600C0E0C0F0C083C082C0D075D000C000C0B2
:0D2EF60001C002C003C004C005C006C00733
:102F030053E8DFADBDAFBEEFFE7C00E42DFFEC3E2A
:102F1300FEADBBED25E02408F582E43402F583EE33
:072F2300F0A3EFF0122C1ED9
:102F2A00D007D006D005D004D003D002D001D000FB
:0B2F3A00D0D0D082D083D0F0D0E032A5
:10211600900222E0FFA3E090028ACFF0A3EFF090B6
:102126000220E0FFA3E090028CCFF0A3EFF0900234
:102136001EE0FFA3E090028ECFF0A3EFF0900281A5
:10214600E0603290028AE0FFA3E0900399CFF0A30B
:10215600EFF090028CE0FFA3E090039BCFF0A3EF9B
:10216600F090028EE0FFA3E090039DCFF0A3EFF086
:10217600E4900281F07F00121DCA7F01121DCA7F02
:1021860002121DCAAD18AC17D374649D74089C5016
:1021960010ED249CFEEC34F7900311F0A3CEF080F2
:1021A60029C3749C9D74079C5012C3ED9464EC94EF
:1021B600085009E4900311F0A3F0800EED2464FEAC
:1021C600EC34F8900311F0A3CEF090021AE0FFA3CE
:1021D600E0900315CFF0A3EFF0900218E0FEA3E025
:1021E600FFEE3395E0FDFCE47B08FAF9F812303493
:1021F600E42FFFEE34FF900317F0A3EFF0900311E6
:10220600E0FEA3E0FFFBAA06EA3395E0F9F89003A7
:1022160015E0FEA3E0FFEE3395E0FDFC121BC29035
:10222600030B121C5CE4FB7A08F9F890030BE0FC44
:10223600A3E0FDA3E0FEA3E0FF12303490030FEE0F
:10224600F0A3EFF0AE19AF1AE4FCFD90031B121CCD
:102256005C900317E0FEA3E0FFEE3395E0FDFC90F3
:10226600031BE0F8A3E0F9A3E0FAA3E0FB121BC20C
:1022760090030B121C5CE4FB7A04F9F890030BE064
:10228600FCA3E0FDA3E0FEA3E0FF123034900313AD
:10229600EEF0A3EFF0AE15AF167C007D09121B45DC
:1022A6007D0C121B57EF24ABFFEE3402FE90031099
:1022B600E02FFF90030FE03E900282F0A3EFF0D3F1
:1022C600E094FF900282E06480948F4007740FF0E0
:1022D600A374FFF0C3900282E0648094805004E40B
:1022E600F0A3F0900282E0FEA3E0FFEE3395E0FD5E
:1022F600FCE4FB7A0DF9F8121BC290030B121C5C6E
:1023060090030BE0FCA3E0FDA3E0FEA3E0FFE4FBEB
:102316007A10F9F812303490030B121C5CE4900327
:102326000FF0A3F0C3900310E0940D90030FE06448
:10233600809480507BA3E025E0FF90030FE033FEFE
:1023460074A72FF58274183EF583E493FF74019306
:10235600900311CFF0A3EFF0900311E0FEA3E0FF8E
:10236600EE3395E0FDFC90030BE0F8A3E0F9A3E063
:10237600FAA3E0FBC3121C11402590030BE0A3E077
:10238600A3E0A3E0FF900311E0A3E0FEEF9E90031D
:1023960019F090030FE0A3E00490031AF080119067
:1023A6000310E004F0700690030FE004F002232A05
:1023B600900319E075F002A424A7F582E5F034161F
:1023C600F583E493FE740193FF90031AE0FDEFA8F2
:1023D60005088005CEC313CE13D8F9FF90023FEE51
:1023E600F0A3EFF0900313E0FEA3E0FF900240E0BD
:0823F6002FF090023FE03EF0E1
:0123FE0022BC
:10334500A2AFE433FDC2AF758F0375B7A575B7F1AD
:0F3355008F828E83E4F0F58FAF05EF24FF92AFE8
:013364002246
:1032E300A2AFE433FCC2AF758F0175B7A575B7F113
:1032F3008F828E83EDF0E4F58FAF04EF24FF92AF5E
:0133030022A7
:102FA20090032CEEF0A3EFF0A3ECF0A3EDF0EB4ACC
:102FB200603990032CE0FEA3E0FFA3E0FCA3E0F560
:102FC200828C83E0FD1232E3EB1B70011A90032F17
:102FD200E004F0700690032EE004F090032DE0046C
:0C2FE200F0700690032CE004F080C32285
:08344E00E4900000F0A3F0225D
:10320D00900000E0FEA3E0FF123345900000E0FEC9
:10321D00A3E0FF7C007D027B007A02122FA2E490D6
:06322D000000F0A3F022F6
:0A2CCF00900326EEF0A3EFF0A90534
:102CD900900326E0FEA3E0EE54FEFE900000E0FC27
:102CE900A3E07002EE6C606B900000E07002A3E05C
:102CF900600312320D900326E0FEA3E0EE54FE902D
:102D09000000F0A3E4F0900000E0FFA3E0900328A6
:102D1900CFF0A3EFF07E007F02A37400F0A374024A
:102D2900F07F007E02EF4E602A900328E475F001DF
:102D3900121BAC85F082F583E493FD90032AE475B8
:102D4900F001121BAC85F082F583EDF0EF1F7001E5
:102D59001E80D2900326E0FCA3E0FDEC5401FC7434
:0B2D6900022DF58274003CF583E9F0B8
:012D7400223C
:102FEE0090031FEEF0A3EFF0A3EBF0A3EAF0A3E93A
:102FFE00F090032474FFF5F0121BAC45F0602690A0
:10300E00031FE475F001121BACAFF0FE900321E03C
:10301E00FBA3E475F001121BACA9F0FA121B1AFD0A
:06302E00122CCF80CC2221
:092ED40046039900000000000013
:0E1DCA0090FFFF121CCBEFF090FFEE121CCB2F
:101DD800851B83851C82E4F0A3F0900012121CEF8F
:101DE800E025E02499F582E43403F583E0FEA3E0DE
:101DF800FFFBAA06E4F9F8900012121CEFE075F058
:101E080002A4248AF582E5F03402F583E0FEA3E01B
:101E1800FFE4C3EF9BFFEE9AFEE499FDE498FC858E
:101E28001B83851C82A3A3121C5CE47F08FEFDFCB7
:101E3800851B83851C82A3A3E0F8A3E0F9A3E0FA3D
:101E4800A3E0FBC3121C11400B851B83851C82E495
:101E5800F0A304F074FF7FF8FEFDFC851B83851C4E
:101E680082A3A3E0F8A3E0F9A3E0FAA3E0FBD3126E
:101E78001C11500B851B83851C8274FFF0A3F08511
:101E88001B83851C82E0FEA3E04E700302210F85B0
:101E98001B83851C82E0FEA3E0F47002EEF460036D
:031EA800021F9E78
:101EAB00900012121CEFE025E02499F582E4340334
:101EBB00F583E0FEA3E0FFE4FCFD90000E121CEFA7
:101ECB00121C5CE47F01FEFDFC90000E121CEFE087
:101EDB00F8A3E0F9A3E0FAA3E0FBC3121C11500D29
:101EEB0090000E121CEF121C6800000001900012F3
:101EFB00121CEFE025E02415F8E6FE08E6FFE4FCF3
:101F0B00FD7BFF7A0FF9F8121BC290000E121CEF2B
:101F1B00E0F8A3E0F9A3E0FAA3E0FB123034900061
:101F2B0006121CEF121C5C900012121CEFE075F0F5
:101F3B0002A4248AF582E5F03402F583E0FEA3E0E7
:101F4B00FFE4FCFD900006121CEFE0F8A3E0F9A300
:101F5B00E0FAA3E0FB121BC290000A121CEF121C4A
:101F6B005CE47BFF7A0FF9F890000A121CEFE0FC9F
:101F7B00A3E0FDA3E0FEA3E0FF12303490001212A9
:101F8B001CEFE025E02415F8A60608A6071233EE91
:101F9B000220DE851B83851C82E0FEA3E064014EDC
:051FAB0060030220DECE
:101FB000900012121CEFE025E02415F8E6FE08E67A
:101FC000FFFBAA06E4C374FF9BFF740F9AFEE49420
:101FD00000FDE49400FCE47BFF7A0FF9F8121BC2C9
:101FE000900006121CEF121C5C900012121CEFE015
:101FF00025E02499F582E43403F583E0FEA3E0FFB5
:10200000FBE4C374FF9BFF740F9EFEE49400FDE4A9
:102010009400FC90000A121CEF121C5CE47F01FE8D
:10202000FDFC90000A121CEFE0F8A3E0F9A3E0FA2F
:10203000A3E0FBC3121C11500D90000A121CEF12FA
:102040001C6800000001900006121CEFC083C082D3
:10205000E0FCA3E0FDA3E0FEA3E0FF90000A121C59
:10206000EFE0F8A3E0F9A3E0FAA3E0FB123034D0EC
:1020700082D083121C5C900012121CEFE075F002FB
:10208000A4248AF582E5F03402F583E0FEA3E0FFA4
:10209000FBE4C374FF9BFF740F9EFEE49400FDE419
:1020A0009400FC900006121CEFE0F8A3E0F9A3E016
:1020B000FAA3E0FB121BC2E47BFF7A0FF9F812309F
:1020C00034C374FF9FFF740F9EFE900012121CEF2A
:0E20D000E025E02415F8A60608A6071233EE58
:1020DE00900012121CEFE075F002A4248AF582E53E
:1020EE00F03402F583E0FEA3E0FF900012121CEF25
:1020FE00E025E02499F582E43403F583EEF0A3EFB6
:01210E00F0E0
:07210F00900013121CCB220B
:053259009002FDEDF004
:10325E009002FE74FF121C29EC4D4E4F601090022E
:0E326E00FDE0121B33740129F9E43AFA80E204
:01327C00222F
:042EDD00410331007C
:1033040090031FEFF0A3EDF07F0A122D7590031FB9
:10331400E0FF122D75900320E0FF122D7512346426
:013324002286
:091A09007F02122D7512346422D3
:0631880012346BEF60271A
:10318E009002F87403F0A37452F01231E39002F837
:10319E00E475F001121BAC85F082F583EFF012346A
:0731AE0071EF70E67F0122C2
:0331B5007F002276
:1030B9009003A3EFF0900331E0FF04F074322FF591
:1030C90082E43403F583742FF0900331E0D3941F25
:1030D9004002E4F07F2F122D759003A3E0FF122D1B
:0530E9007512346422A1
:1030EE009003A4EFF0900331E0FF04F074322FF55B
:1030FE0082E43403F5837430F0900331E0D3941FEF
:10310E004002E4F07F30122D759003A4E0FF122DE3
:05311E0075123464226B
:011A1500FFD1
:022EE100C10F1F
:102F4500E49002F9F0FB7A0079149002FE121C68F5
:102F550000000007E4FD12325975170875180012B4
:102F6500344EE49002F8F09002F8E0C3941E502924
:102F7500E075F007A42400F582E4343AAF82FE7BC5
:102F8500007A007914900324E4F0A37407F0122F5B
:0C2F9500EE9002F8E004F080CE12320D45
:012FA100220D
:1033EE00200B04D20BD20A200F06300903121A0941
:0333FE00D20F22C9
:1033BD00901A15E493600C122F457E1A7F15E4FDCB
:0933CD001232E3E49003A5F022A2
:1032A0009003A5E075F007A42400F9743A35F0FA0C
:1032B0007BFF78147C007D007E007F07121AF4C229
:0232C0000F22DB
:1031B80012344E9003A5E075F007A42400F582E4CC
:1031C800343AAF82FE7B007A007914900324E4F04D
:0B31D800A37407F0122FEE12320D223C
:061A1B001231B8C20F22D7
:0826130090036AEFF0A3EDF063
:10261B0090036AE0D39B50030226F8E024FFFEE40C
:10262B0034FF90036FF0A3CEF0EB1490036EF09099
:10263B00036BE024FFFFE434FFFED3900370E09FB5
:10264B00EE6480F890036FE064809840030227CE1D
:10265B00E0FEA3E0903A0075F007121C99EE75F0BE
:10266B0007A42583AF82900376F0A3EFF090036E5F
:10267B00E075F007A42400F9743A35F0FA9003736F
:10268B0074FFF0A3EAF0A3E9F0E4900371F0A3F078
:10269B00C3900372E09407900371E0940050349060
:1026AB000373E0A3E475F001121BACFEAFF09003D3
:1026BB0076E475F001121BAC85F082F583E493FD93
:1026CB00122CCF900372E004F07006900371E004BB
:1026DB00F080BD12320D900370E004F07006900391
:1026EB006FE004F090036EE004F002263A90036B67
:1026FB00E024FFFEE434FF90036FF0A3CEF09003D1
:10270B006DE014A3F090036AE024FFFFE434FFFEB6
:10271B00C3900370E09FEE6480F890036FE06480D9
:10272B009850030227CEE0FEA3E0903A0075F00725
:10273B00121C99EE75F007A42583AF82900376F0F7
:10274B00A3EFF090036EE075F007A42400F9743A40
:10275B0035F0FA90037374FFF0A3EAF0A3E9F0E409
:10276B00900371F0A3F0C3900372E0940790037190
:10277B00E094005034900373E0A3E475F001121B56
:10278B00ACFEAFF0900376E475F001121BAC85F054
:10279B0082F583E493FD122CCF900372E004F0706A
:1027AB0006900371E004F080BD12320D900370E0CF
:1027BB0024FFF090036FE034FFF090036EE014F011
:0327CB00022710D2
:0127CE0022E8
:0527CF00900359EDF03C
:1027D400EF14900366F0EB14A3F0900359E014FF98
:1027E400900366E0D39F4003022938A3E075F00705
:1027F400A42400F582E4343AAF82FEE4900368F046
:10280400A3F0C3900369E09407900368E094005038
:10281400300FEFAC0670010E14F5828C83E493FD47
:10282400900368E0A3E0245FF582E43403F583EDCC
:10283400F0900369E004F07006900368E004F0800F
:10284400C1900367E075F007A42400F9743A35F0E9
:10285400FA90035A74FFF0A3EAF0A3E9F090036638
:10286400E075F007A42400F582E4343AAF829003C3
:102874005DF0A3EFF0E4900368F0A3F0C390036964
:10288400E09407900368E09400503490035AE0A366
:10289400E475F001121BACFEAFF090035DE475F03B
:1028A40001121BAC85F082F583E493FD122CCF90CA
:1028B4000369E004F07006900368E004F080BD90C2
:1028C4000366E075F007A42400F9743A35F0FA9031
:1028D400035A74FFF0A3EAF0A3E9F0E4900368F06C
:1028E400A3F0C3900369E09407900368E094005058
:1028F4003390035AE0A3E475F001121BACFEAFF071
:10290400900368E0A3E0245FF582E43403F583E0F8
:10291400FD122CCF900369E004F07006900368E088
:1029240004F080BE12320D900366E004F0A3E004CC
:04293400F00227DEA8
:01293800227C
:0B2B3100900378EFF0A3EDF0A3EBF0B1
:102B3C00A3E5C1F0A2AFE433A3F0900379E0FF90DA
:102B4C00037DE4F0A3EFF0E0F8E4F0E890037DF00F
:102B5C00900378E0FF90037DE0F0A3E04FF0C2AF6C
:102B6C00900380740FF0900380E0C3941E40030226
:102B7C002C0E12344E900380E075F007A42400F95B
:102B8C00743A35F0FA90038274FFF0A3EAF0A3E9EB
:102B9C00F0E490037FF090037FE0C39407505790CC
:102BAC00037DE0A3E0900378F090037DE09003793F
:102BBC00F0900378E0FFA3E0FDA3E0FBE490039525
:102BCC00F0D2001218C3900381EFF0A3E0A3E475D8
:102BDC00F001121BACFEAFF0900381E0FD122CCF84
:102BEC0090037EE004F0700690037DE004F0900307
:102BFC007FE004F080A012320D900380E004F0021C
:102C0C002B7290037BE0F5C1A3E024FF92AF12344A
:012C1C006453
:012C1D002294
:0B293900900385EFF0A3EDF0A3EBF09E
:10294400A3E5C1F0A2AFE433A3F0900386E0FF90C7
:10295400038EE4F0A3EFF0E0F8E4F0E890038EF0E7
:10296400900385E0FF90038EE0F0A3E04FF0C2AF48
:1029740090038CE4F0A3740FF0C390038DE0941ED5
:1029840090038CE094004003022A28E0FEA3E09028
:102994003A0075F007121C99EE75F007A42583AF71
:1029A40082900390F0A3EFF0E490038AF0A3F0C3C5
:1029B40090038BE0940790038AE0940050559003B1
:1029C4008EE0A3E0900385F090038EE0900386F000
:1029D400900385E0FFA3E0FDA3E0FB900390E47582
:1029E400F001121BAC85F082F583E493900395F01B
:1029F400C2001218C390038FE004F0700690038E97
:102A0400E004F090038BE004F0700690038AE00485
:102A1400F0809C90038DE004F0700690038CE00439
:102A2400F002297D900388E0F5C1A3E024FF92AF72
:032A3400123464F5
:012A3700227C
:0818C300900392EFF0A3EDF099
:1018CB00A2009204C2062010FDD210900396EBF0FA
:1018DB00C201D202D2057F01C2C4C207D2C530C039
:1018EB00FDE5C054F02480700302197D24C0601BF9
:1018FB0024E060030219AD900396E0F5C2A201E467
:10190B003342C2C2C5E4A3F00219AF30C15930074C
:10191B0007D2C5C2070219AF30020CC202D2039024
:10192B000393E0F5C2807D300311C203900392E074
:10193B00F5C230046FD207D2018069200166EFFD3A
:10194B00900397E0FB3395E0FAC3EB9D7480F86A44
:10195B0098500E900395E0F5C2900397E004F08049
:10196B0043D2C4C210803D300504D2C58036D206A6
:10197B008032EFFD900397E0FB3395E0FAC3EB9DCC
:10198B007480F86A98500CA3E5C2F0900397E004BA
:10199B00F0D2C1900397E0B5070AC210C2C1D2C4FE
:1019AB008002D20630060853C0BF43C040C210C2EB
:0C19BB00C03010030218E9900398E0FF10
:0119C70022FD
:022EE300C10D1F
:1033D600E50BB50FFBE50AB50EF6E50BB513F1E502
:0833E6000AB512EC20C5E92232
:0F343500438E08758DAF758D5D858D8BD28E2280
:1034130075C101E4F5C2F5C053C17F43C1801234C5
:02342300352250
:103233007E027F988E0C8F0D8E108F118E088F0952
:103243007E027FC88E0E8F0F8E128F138E0A8F0B06
:06325300C20C123413222C
:103123000511E511AA107002051014F5828A83EFC8
:10313300F0AF050511E511AC107002051014F5820E
:103143008C83EFF074C8B5110B7402B510067510BB
:05315300027511982235
:07346400C20CC2C4D2C52254
:102D7500200C45D20C0513E513AC12700205121494
:102D8500F5828C8374FFF074F8B5130B7402B512D9
:102D9500067512027513C80513E513AC127002050A
:102DA5001214F5828C83E4F074F8B5130B7402B534
:102DB50012067512027513C80513E513AC127002DD
:102DC500051214F5828C83E4F074F8B5130B7402C4
:102DD500B512067512027513C80513E513AC12700A
:102DE50002051214F5828C83EFF074F8B5130B7499
:0D2DF50002B512067512027513C87F012287
:10336500AE07E509B50D08E508B50C037F00228514
:0F3375000D82850C83E0B506037F01227F0022C5
:1031E300050DE50D7002050C050DE50DAE0C700225
:1031F300050C14F5828E83E0FF74C8B50D0B7402C1
:09320300B50C06750C02750D985E
:01320C00229F
:06346B007FFF1233652211
:06347100E4FF12336522A6
:031A18000223FFA7
:1023FF00C0E0C083C082C0D075D000C000C002C092
:07240F0004C005C006C00770
:10241600E5C054FE121CA525DA0825DA0A25F00CBB
:1024260025F00E25B91025B91225CC1425CC162574
:10243600B11C25B11E25AD2425AD262553282553CF
:102446002A257C2C257C2E253842254144254146CB
:10245600254A50254A52254A54254A56252F88256D
:102466002F8A24BAC024C7C22478E02478E2000068
:1024760025FCC2C5050BE50B7002050AB4F80B7402
:1024860002B50A06750A02750BC8050BE50BAE0AFE
:102496007002050A14F5828E83E0F5C274F8650BA6
:1024A60070047402650A60030225FC750A02750B46
:1024B600C80225FC850E0A850F0BD2C4D2C502259B
:1024C600FCE50BB51312E50AB5120D85120E851340
:1024D6000FC2C5D2C40225FC850B82850A83E0B4EF
:1024E600FF07C2C4D2C50225FC050BE50B70020529
:1024F6000AB4F80B7402B50A06750A02750BC8050C
:102506000BE50BAE0A7002050A14F5828E83E0F520
:10251600C274F8650B70047402650A60030225FC38
:10252600750A02750BC80225FC900330E004F00220
:1025360025FC900330E004F00225FC900330E00413
:10254600F00225FC900330E004F00225FCE5C260B1
:1025560013900286E065C2600BC2C4C2C5C2C1C286
:102566000E0225FCADC27FFF123123C2C4C2C5D202
:10257600C1D20E0225FC850E0A850F0BC2C5D20DEF
:10258600E5C26012900286E065C2600AC2C4C2C596
:10259600C2C1C20E8060ADC27FFF123123C2C4C267
:1025A600C5D2C1D20E804FD2C5804B850A0E850B8F
:1025B6000F8043851008851109C2C4C2C1300D368B
:1025C600D2C5C20D8030850E0A850F0BC2C4C2C1AA
:1025D600D2C58022C2C4C2C5200E04C2C18017ADB6
:1025E600C2E4FF123123D2C1800C850E0A850F0B7F
:0825F600C2C1C2C4D2C5C2C0BB
:1025FE00D007D006D005D004D002D000D0D0D082E3
:05260E00D083D0E03292
:10062700022E02E493A3F8E493A34003F68001F2B9
:1006370008DFF48029E493A3F85407240CC8C333D4
:10064700C4540F4420C8834004F456800146F6DFA3
:10065700E4800B0102040810204080902E7CE47E89
:10066700019360BCA3FF543F30E509541FFEE49398
:10067700A360010ECF54C025E060A840B8E493A35F
:10068700FAE493A3F8E493A3C8C582C8CAC583CA8A
:10069700F0A3C8C582C8CAC583CADFE9DEE780BE42
:012EE50000EC
:101A2400E709F608DFFA8046E709F208DFFA803EA4
:101A340088828C83E709F0A3DFFA8032E309F60891
:101A4400DFFA8078E309F208DFFA807088828C83F9
:101A5400E309F0A3DFFA806489828A83E0A3F608AD
:101A6400DFFA805889828A83E0A3F208DFFA804C87
:101A740080D280FA80C680D4806980F2803380105E
:101A840080A680EA809A80A880DA80E280CA8033C7
:101A940089828A83ECFAE493A3C8C582C8CCC5833F
:101AA400CCF0A3C8C582C8CCC583CCDFE9DEE7800F
:101AB4000D89828A83E493A3F608DFF9ECFAA9F08E
:101AC400EDFB2289828A83ECFAE0A3C8C582C8CCE4
:101AD400C583CCF0A3C8C582C8CCC583CCDFEADEFD
:101AE400E880DB89828A83E493A3F208DFF980CC5F
:101AF40088F0EF60010E4E60C388F0ED2402B40458
:101B04000050B9F582EB2402B4040050AF232345FE
:061B14008223901A747395
:101B1A00BB010689828A83E0225002E722BBFE02C9
:091B2A00E32289828A83E49322FC
:101B3300BB010689828A83F0225002F722BBFE0191
:021B4300F3228B
:101B4500EF8DF0A4A8F0CF8CF0A428CE8DF0A42EB4
:021B5500FE226E
:101B5700BC000BBE0029EF8DF084FFADF022E4CC72
:101B6700F875F008EF2FFFEE33FEEC33FCEE9DEC3B
:101B7700984005FCEE9DFE0FD5F0E9E4CEFD22ED81
:101B8700F8F5F0EE8420D21CFEADF075F008EF2FCB
:101B9700FFED33FD4007985006D5F0F222C398FDBC
:051BA7000FD5F0EA2259
:101BAC00A3F8E0C5F025F0F0E582158270021583EC
:061BBC00E0C838F0E82249
:101BC200E88FF0A4CC8BF0A42CFCE98EF0A42CFCC2
:101BD2008AF0EDA42CFCEA8EF0A4CDA8F08BF0A440
:101BE2002DCC3825F0FDE98FF0A42CCD35F0FCEB9F
:101BF2008EF0A4FEA9F0EB8FF0A4CFC5F02ECD3964
:0F1C0200FEE43CFCEAA42DCE35F0FDE43CFC22D0
:10303400C2D5E830E70FB2D5E4C39BFBE49AFAE4C7
:1030440099F9E498F8EC30E717B2D512306A121DFA
:1030540038E4C39BFBE49AFAE499F9E498F8800312
:10306400121D3830D50DE4C39FFFE49EFEE49DFDA0
:04307400E49CFC22BA
:101C1100EB9FF5F0EA9E42F0E99D42F0EC6480C84A
:061C210064809845F022EA
:101C27007401FF3395E0FEFDFCA3A3A3E0CF2FF0E3
:101C3700E582158270021583E0CE3EF0E5821582BB
:101C470070021583E0CD3DF0E582158270021583A1
:051C5700E0CC3CF0228E
:0C1C5C00ECF0A3EDF0A3EEF0A3EFF022FB
:101C6800A8828583F0D083D082121C7F121C7F1239
:101C78001C7F121C7FE473E493A3C583C5F0C5835E
:101C8800C8C582C8F0A3C583C5F0C583C8C582C8C6
:011C98002229
:0C1C9900A42582F582E5F03583F5832256
:101CA500D083D082F8E4937012740193700DA3A3CE
:101CB50093F8740193F5828883E4737402936860E2
:061CC500EFA3A3A380DFE2
:101CCB00E51C2582F582E51B3583F583B51B048561
:101CDB00821C2210AF0685821CF51B2285821CF507
:041CEB001BD2AF2237
:0D1CEF00E51C2582F582E51B3583F5832277
:101CFC0075F008758200EF2FFFEE33FECD33CDCC9F
:101D0C0033CCC58233C5829BED9AEC99E582984021
:101D1C000CF582EE9BFEED9AFDEC99FC0FD5F0D6FE
:101D2C00E4CEFBE4CDFAE4CCF9A88222B800C1B928
:101D3C000059BA002DEC8BF084CFCECDFCE5F0CB66
:101D4C00F97818EF2FFFEE33FEED33FDEC33FCEB9F
:101D5C0033FB10D703994004EB99FB0FD8E5E4F95A
:101D6C00FA227818EF2FFFEE33FEED33FDEC33FC47
:101D7C00C933C910D7059BE99A4007EC9BFCE99A3B
:101D8C00F90FD8E0E4C9FAE4CCFB2275F010EF2F80
:101D9C00FFEE33FEED33FDCC33CCC833C810D70780
:101DAC009BEC9AE899400AED9BFDEC9AFCE899F8BB
:0E1DBC000FD5F0DAE4CDFBE4CCFAE4C8F9224E
:00000001FF
